BL51 BANKED LINKER/LOCATER V6.22                                                        08/01/2023  15:50:03  PAGE 1


BL51 BANKED LINKER/LOCATER V6.22, INVOKED BY:
D:\KEIL\C51\BIN\BL51.EXE .\Objects\STARTUP.obj, .\Objects\GPIO.obj, .\Objects\Initial.obj, .\Objects\main.obj, .\Objects
>> \Touch_Lib.obj, .\Objects\TouchKeyScan.obj, .\User\C\XC8FT8463_Touch_TEST.LIB TO .\Objects\XC8FT8463 PRINT (.\Listing
>> s\XC8FT8463.m51) RAMSIZE (256)


MEMORY MODEL: SMALL


INPUT MODULES INCLUDED:
  .\Objects\STARTUP.obj (?C_STARTUP)
  .\Objects\GPIO.obj (GPIO)
  .\Objects\Initial.obj (INITIAL)
  .\Objects\main.obj (MAIN)
  .\Objects\Touch_Lib.obj (TOUCH_LIB)
  .\Objects\TouchKeyScan.obj (TOUCHKEYSCAN)
  D:\KEIL\C51\LIB\C51S.LIB (?C_INIT)
  D:\KEIL\C51\LIB\C51S.LIB (?C?CLDPTR)
  D:\KEIL\C51\LIB\C51S.LIB (?C?CLDOPTR)
  D:\KEIL\C51\LIB\C51S.LIB (?C?CILDOPTR)
  D:\KEIL\C51\LIB\C51S.LIB (?C?CSTPTR)
  D:\KEIL\C51\LIB\C51S.LIB (?C?CSTOPTR)
  D:\KEIL\C51\LIB\C51S.LIB (?C?SIDIV)
  D:\KEIL\C51\LIB\C51S.LIB (?C?ILDOPTR)
  D:\KEIL\C51\LIB\C51S.LIB (?C?ISTPTR)
  D:\KEIL\C51\LIB\C51S.LIB (?C?ISTOPTR)
  D:\KEIL\C51\LIB\C51S.LIB (?C?ULDIV)
  D:\KEIL\C51\LIB\C51S.LIB (?C?LLDPTR)
  D:\KEIL\C51\LIB\C51S.LIB (?C?LLDOPTR)
  D:\KEIL\C51\LIB\C51S.LIB (?C?LSTPTR)
  D:\KEIL\C51\LIB\C51S.LIB (?C?LLDPTR0)
  D:\KEIL\C51\LIB\C51S.LIB (?C?LSTKOPTR)
  D:\KEIL\C51\LIB\C51S.LIB (?C?OFFXADD)
  D:\KEIL\C51\LIB\C51S.LIB (?C?UIDIV)
  D:\KEIL\C51\LIB\C51S.LIB (?C?LLDIDATA)
  D:\KEIL\C51\LIB\C51S.LIB (?C?LLDXDATA)
  D:\KEIL\C51\LIB\C51S.LIB (?C?LLDPDATA)
  D:\KEIL\C51\LIB\C51S.LIB (?C?LLDCODE)
  D:\KEIL\C51\LIB\C51S.LIB (?C?LLDIDATA0)
  D:\KEIL\C51\LIB\C51S.LIB (?C?LLDXDATA0)
  D:\KEIL\C51\LIB\C51S.LIB (?C?LLDPDATA0)
  D:\KEIL\C51\LIB\C51S.LIB (?C?LLDCODE0)
  D:\KEIL\C51\LIB\C51S.LIB (?C?LSTIDATA)
  D:\KEIL\C51\LIB\C51S.LIB (?C?LSTXDATA)
  D:\KEIL\C51\LIB\C51S.LIB (?C?LSTPDATA)
  D:\KEIL\C51\LIB\C51S.LIB (?C?LSTKIDATA)
  D:\KEIL\C51\LIB\C51S.LIB (?C?LSTKXDATA)
  D:\KEIL\C51\LIB\C51S.LIB (?C?LSTKPDATA)


LINK MAP OF MODULE:  .\Objects\XC8FT8463 (?C_STARTUP)


            TYPE    BASE      LENGTH    RELOCATION   SEGMENT NAME
            -----------------------------------------------------

            * * * * * * *   D A T A   M E M O R Y   * * * * * * *
            REG     0000H     0008H     ABSOLUTE     "REG BANK 0"
BL51 BANKED LINKER/LOCATER V6.22                                                      08/01/2023  15:50:03  PAGE 2


            DATA    0008H     0017H     UNIT         _DATA_GROUP_
            DATA    001FH     0014H     UNIT         ?DT?TOUCH_LIB
            IDATA   0033H     0001H     UNIT         ?STACK

            * * * * * * *  X D A T A   M E M O R Y  * * * * * * *
            XDATA   0000H     0086H     UNIT         ?XD?TOUCHKEYSCAN
            XDATA   0086H     0032H     UNIT         ?XD?TOUCH_LIB

            * * * * * * *   C O D E   M E M O R Y   * * * * * * *
            CODE    0000H     0003H     ABSOLUTE     
            CODE    0003H     002AH     UNIT         ?PR?MAIN?MAIN
            CODE    002DH     0003H     UNIT         ?PR?DELAY_US?TOUCH_LIB
                    0030H     0003H                  *** GAP ***
            CODE    0033H     0003H     ABSOLUTE     
            CODE    0036H     0026H     UNIT         ?PR?TKL_CSDINIT?TOUCH_LIB
                    005CH     0007H                  *** GAP ***
            CODE    0063H     0003H     ABSOLUTE     
            CODE    0066H     0435H     UNIT         ?C?LIB_CODE
            CODE    049BH     0275H     UNIT         ?PR?_THRESHOLDINIT?TOUCH_LIB
            CODE    0710H     0209H     UNIT         ?PR?_TKL_KEY_FINDICOMTREATMENT?TOUCH_LIB
            CODE    0919H     01BDH     UNIT         ?PR?_GPIO_SET_MODE?TOUCH_LIB
            CODE    0AD6H     0118H     UNIT         ?PR?_TKL_ADDDATATOBUF?TOUCH_LIB
            CODE    0BEEH     0110H     UNIT         ?PR?_TKL_INIT?TOUCH_LIB
            CODE    0CFEH     00FAH     UNIT         ?PR?_TKL_ACQUISITION?TOUCH_LIB
            CODE    0DF8H     00D9H     UNIT         ?C_INITSEG
            CODE    0ED1H     00C9H     UNIT         ?PR?TKL_PROCESSALL?TOUCH_LIB
            CODE    0F9AH     0092H     UNIT         ?PR?_TKL_KEY_SETFINDICOMSTATE?TOUCH_LIB
            CODE    102CH     0090H     UNIT         ?PR?TKL_IRQCALLBACK?TOUCH_LIB
            CODE    10BCH     008CH     UNIT         ?C_C51STARTUP
            CODE    1148H     0073H     UNIT         ?PR?_TKL_KEY_SETCALIBRATIONSTATE?TOUCH_LIB
            CODE    11BBH     005FH     UNIT         ?PR?_TKL_KEY_SETERRORSTATE?TOUCH_LIB
            CODE    121AH     005DH     UNIT         ?PR?I2C_WRITE_BUFFER?TOUCH_LIB
            CODE    1277H     0058H     UNIT         ?PR?INITIAL_TRIM?INITIAL
            CODE    12CFH     0051H     UNIT         ?PR?TKL_SCANSTARTLOOP?TOUCH_LIB
            CODE    1320H     004CH     UNIT         ?PR?GPIO_INIT?GPIO
            CODE    136CH     0044H     UNIT         ?PR?TIMER0_IRQHANDLER?TOUCHKEYSCAN
            CODE    13B0H     003BH     UNIT         ?PR?CSD_IRQHANDLER?TOUCHKEYSCAN
            CODE    13EBH     0035H     UNIT         ?PR?IIC_WAIT_ACK?TOUCH_LIB
            CODE    1420H     0032H     UNIT         ?PR?_IIC_SEND_BYTE?TOUCH_LIB
            CODE    1452H     0032H     UNIT         ?PR?TKL_ACQUISITIONALL?TOUCH_LIB
            CODE    1484H     001AH     UNIT         ?PR?_DELAYMS?INITIAL
            CODE    149EH     0018H     UNIT         ?PR?TKL_ACTION?TOUCH_LIB
            CODE    14B6H     0018H     UNIT         ?CO?TOUCHKEYSCAN
            CODE    14CEH     0016H     UNIT         ?PR?SYSTEM_INIT?INITIAL
            CODE    14E4H     0016H     UNIT         ?PR?SDA_OUT?TOUCH_LIB
            CODE    14FAH     0016H     UNIT         ?PR?SDA_IN?TOUCH_LIB
            CODE    1510H     0016H     UNIT         ?PR?IIC_STOP?TOUCH_LIB
            CODE    1526H     0014H     UNIT         ?PR?I2C_INIT?TOUCH_LIB
            CODE    153AH     0014H     UNIT         ?PR?IIC_START?TOUCH_LIB
            CODE    154EH     0010H     UNIT         ?PR?TIMER0_INIT?TOUCHKEYSCAN
            CODE    155EH     000EH     UNIT         ?PR?_DELAY_US1?TOUCH_LIB



OVERLAY MAP OF MODULE:   .\Objects\XC8FT8463 (?C_STARTUP)


BL51 BANKED LINKER/LOCATER V6.22                                                      08/01/2023  15:50:03  PAGE 3


SEGMENT                                            DATA_GROUP 
  +--> CALLED SEGMENT                            START    LENGTH
----------------------------------------------------------------
?C_C51STARTUP                                    -----    -----
  +--> ?PR?MAIN?MAIN
  +--> ?C_INITSEG

?PR?MAIN?MAIN                                    -----    -----
  +--> ?PR?SYSTEM_INIT?INITIAL
  +--> ?PR?GPIO_INIT?GPIO
  +--> ?PR?TIMER0_INIT?TOUCHKEYSCAN
  +--> ?CO?TOUCHKEYSCAN
  +--> ?PR?_TKL_INIT?TOUCH_LIB
  +--> ?PR?TKL_ACTION?TOUCH_LIB

?PR?SYSTEM_INIT?INITIAL                          -----    -----
  +--> ?PR?_DELAYMS?INITIAL
  +--> ?PR?INITIAL_TRIM?INITIAL

?PR?_TKL_INIT?TOUCH_LIB                          0008H    0011H
  +--> ?PR?I2C_INIT?TOUCH_LIB
  +--> ?PR?_THRESHOLDINIT?TOUCH_LIB
  +--> ?PR?_TKL_KEY_SETFINDICOMSTATE?TOUCH_LIB
  +--> ?PR?TKL_CSDINIT?TOUCH_LIB

?PR?_THRESHOLDINIT?TOUCH_LIB                     0019H    0004H

?PR?_TKL_KEY_SETFINDICOMSTATE?TOUCH_LIB          0019H    0001H

?PR?TKL_ACTION?TOUCH_LIB                         -----    -----
  +--> ?PR?TKL_ACQUISITIONALL?TOUCH_LIB
  +--> ?PR?TKL_PROCESSALL?TOUCH_LIB

?PR?TKL_ACQUISITIONALL?TOUCH_LIB                 0008H    0001H
  +--> ?PR?_TKL_ACQUISITION?TOUCH_LIB

?PR?_TKL_ACQUISITION?TOUCH_LIB                   0009H    000FH

?PR?TKL_PROCESSALL?TOUCH_LIB                     0008H    0001H
  +--> ?PR?_TKL_KEY_FINDICOMTREATMENT?TOUCH_LIB
  +--> ?PR?I2C_WRITE_BUFFER?TOUCH_LIB

?PR?_TKL_KEY_FINDICOMTREATMENT?TOUCH_LIB         0009H    0005H
  +--> ?PR?_TKL_KEY_SETERRORSTATE?TOUCH_LIB
  +--> ?PR?_TKL_KEY_SETCALIBRATIONSTATE?TOUC...

?PR?_TKL_KEY_SETERRORSTATE?TOUCH_LIB             000EH    0001H

?PR?_TKL_KEY_SETCALIBRATIONSTATE?TOUC...         000EH    0001H

?PR?I2C_WRITE_BUFFER?TOUCH_LIB                   -----    -----
  +--> ?PR?IIC_START?TOUCH_LIB
  +--> ?PR?_IIC_SEND_BYTE?TOUCH_LIB
  +--> ?PR?IIC_STOP?TOUCH_LIB

?PR?IIC_START?TOUCH_LIB                          -----    -----
  +--> ?PR?SDA_OUT?TOUCH_LIB
BL51 BANKED LINKER/LOCATER V6.22                                                      08/01/2023  15:50:03  PAGE 4


  +--> ?PR?_DELAY_US1?TOUCH_LIB

?PR?_IIC_SEND_BYTE?TOUCH_LIB                     -----    -----
  +--> ?PR?SDA_OUT?TOUCH_LIB
  +--> ?PR?DELAY_US?TOUCH_LIB
  +--> ?PR?_DELAY_US1?TOUCH_LIB
  +--> ?PR?IIC_WAIT_ACK?TOUCH_LIB

?PR?IIC_WAIT_ACK?TOUCH_LIB                       -----    -----
  +--> ?PR?SDA_IN?TOUCH_LIB
  +--> ?PR?DELAY_US?TOUCH_LIB
  +--> ?PR?_DELAY_US1?TOUCH_LIB
  +--> ?PR?IIC_STOP?TOUCH_LIB
  +--> ?PR?SDA_OUT?TOUCH_LIB

?PR?IIC_STOP?TOUCH_LIB                           -----    -----
  +--> ?PR?SDA_OUT?TOUCH_LIB
  +--> ?PR?_DELAY_US1?TOUCH_LIB
  +--> ?PR?DELAY_US?TOUCH_LIB

*** NEW ROOT ***************************************************

?PR?TIMER0_IRQHANDLER?TOUCHKEYSCAN               -----    -----
  +--> ?PR?TKL_SCANSTARTLOOP?TOUCH_LIB

*** NEW ROOT ***************************************************

?PR?CSD_IRQHANDLER?TOUCHKEYSCAN                  -----    -----
  +--> ?PR?TKL_IRQCALLBACK?TOUCH_LIB

?PR?TKL_IRQCALLBACK?TOUCH_LIB                    -----    -----
  +--> ?PR?_GPIO_SET_MODE?TOUCH_LIB
  +--> ?PR?_TKL_ADDDATATOBUF?TOUCH_LIB

?PR?_TKL_ADDDATATOBUF?TOUCH_LIB                  001DH    0002H



SYMBOL TABLE OF MODULE:  .\Objects\XC8FT8463 (?C_STARTUP)

  VALUE           TYPE          NAME
  ----------------------------------

  -------         MODULE        ?C_STARTUP
  C:10BCH         SEGMENT       ?C_C51STARTUP
  I:0033H         SEGMENT       ?STACK
  C:0000H         PUBLIC        ?C_STARTUP
  D:00E0H         SYMBOL        ACC
  D:00F0H         SYMBOL        B
  D:0083H         SYMBOL        DPH
  D:0082H         SYMBOL        DPL
  N:0000H         SYMBOL        IBPSTACK
  N:0100H         SYMBOL        IBPSTACKTOP
  N:0080H         SYMBOL        IDATALEN
  C:10BFH         SYMBOL        IDATALOOP
  N:0000H         SYMBOL        PBPSTACK
  N:0100H         SYMBOL        PBPSTACKTOP
BL51 BANKED LINKER/LOCATER V6.22                                                      08/01/2023  15:50:03  PAGE 5


  N:0000H         SYMBOL        PDATALEN
  N:0000H         SYMBOL        PDATASTART
  N:0000H         SYMBOL        PPAGE
  N:0000H         SYMBOL        PPAGEENABLE
  D:00A0H         SYMBOL        PPAGE_SFR
  D:0081H         SYMBOL        SP
  C:10BCH         SYMBOL        STARTUP1
  N:0000H         SYMBOL        XBPSTACK
  N:0000H         SYMBOL        XBPSTACKTOP
  N:0000H         SYMBOL        XDATALEN
  N:0000H         SYMBOL        XDATASTART
  C:0000H         LINE#         126
  C:10BCH         LINE#         133
  C:10BEH         LINE#         134
  C:10BFH         LINE#         135
  C:10C0H         LINE#         136
  C:10C2H         LINE#         185
  C:10C5H         LINE#         196
  -------         ENDMOD        ?C_STARTUP

  -------         MODULE        GPIO
  C:0000H         SYMBOL        _ICE_DUMMY_
  D:00A8H         PUBLIC        IE
  C:1320H         PUBLIC        GPIO_Init
  D:00E0H         PUBLIC        ACC
  D:00F8H         PUBLIC        SLPTIM_CR
  D:0080H         PUBLIC        P0_DR
  D:0090H         PUBLIC        P1_DR
  D:00A0H         PUBLIC        P2_DR
  D:00B0H         PUBLIC        P3_DR
  D:00D0H         PUBLIC        PSW
  -------         PROC          GPIO_INIT
  C:1320H         LINE#         11
  C:1320H         LINE#         12
  C:1320H         LINE#         31
  C:1325H         LINE#         32
  C:1329H         LINE#         33
  C:132BH         LINE#         34
  C:132DH         LINE#         35
  C:132FH         LINE#         36
  C:1333H         LINE#         38
  C:1337H         LINE#         39
  C:133BH         LINE#         40
  C:133DH         LINE#         41
  C:133FH         LINE#         42
  C:1341H         LINE#         43
  C:1345H         LINE#         45
  C:1349H         LINE#         46
  C:134DH         LINE#         47
  C:134FH         LINE#         48
  C:1351H         LINE#         49
  C:1353H         LINE#         50
  C:1357H         LINE#         52
  C:135BH         LINE#         53
  C:135DH         LINE#         54
  C:135FH         LINE#         55
  C:1361H         LINE#         56
BL51 BANKED LINKER/LOCATER V6.22                                                      08/01/2023  15:50:03  PAGE 6


  C:1365H         LINE#         58
  C:136BH         LINE#         59
  -------         ENDPROC       GPIO_INIT
  -------         ENDMOD        GPIO

  -------         MODULE        INITIAL
  C:0000H         SYMBOL        _ICE_DUMMY_
  C:14CEH         PUBLIC        System_Init
  D:00A8H         PUBLIC        IE
  D:0095H         PUBLIC        PCLK_CR
  C:1484H         PUBLIC        _DelayMs
  D:00E0H         PUBLIC        ACC
  D:0094H         PUBLIC        CLK_CR
  D:00F8H         PUBLIC        SLPTIM_CR
  C:1277H         PUBLIC        Initial_trim
  D:0080H         PUBLIC        P0_DR
  D:0090H         PUBLIC        P1_DR
  D:00A0H         PUBLIC        P2_DR
  D:00B0H         PUBLIC        P3_DR
  D:00D0H         PUBLIC        PSW
  -------         PROC          _DELAYMS
  D:0006H         SYMBOL        ms
  -------         DO            
  D:0004H         SYMBOL        a
  -------         ENDDO         
  C:1484H         LINE#         9
  C:1484H         LINE#         10
  C:1484H         LINE#         12
  C:1488H         LINE#         13
  C:1488H         LINE#         14
  C:148CH         LINE#         15
  C:1496H         LINE#         16
  C:149BH         LINE#         17
  C:149DH         LINE#         19
  -------         ENDPROC       _DELAYMS
  -------         PROC          INITIAL_TRIM
  -------         DO            
  D:0007H         SYMBOL        temp
  -------         ENDDO         
  C:1277H         LINE#         27
  C:1277H         LINE#         28
  C:1277H         LINE#         31
  C:127CH         LINE#         32
  C:127EH         LINE#         33
  C:1284H         LINE#         34
  C:1288H         LINE#         35
  C:128CH         LINE#         37
  C:1292H         LINE#         38
  C:1298H         LINE#         39
  C:129CH         LINE#         40
  C:12A0H         LINE#         42
  C:12A6H         LINE#         43
  C:12ACH         LINE#         44
  C:12B0H         LINE#         45
  C:12B4H         LINE#         47
  C:12BAH         LINE#         48
  C:12C0H         LINE#         49
BL51 BANKED LINKER/LOCATER V6.22                                                      08/01/2023  15:50:03  PAGE 7


  C:12C4H         LINE#         50
  C:12C8H         LINE#         51
  C:12CEH         LINE#         52
  -------         ENDPROC       INITIAL_TRIM
  -------         PROC          SYSTEM_INIT
  C:14CEH         LINE#         60
  C:14CEH         LINE#         61
  C:14CEH         LINE#         62
  C:14D4H         LINE#         67
  C:14D7H         LINE#         80
  C:14DAH         LINE#         108
  C:14E1H         LINE#         109
  -------         ENDPROC       SYSTEM_INIT
  -------         ENDMOD        INITIAL

  -------         MODULE        MAIN
  C:0000H         SYMBOL        _ICE_DUMMY_
  D:00A8H         PUBLIC        IE
  C:0003H         PUBLIC        main
  D:00E0H         PUBLIC        ACC
  D:00F8H         PUBLIC        SLPTIM_CR
  B:00A8H.7       PUBLIC        IE_EA
  D:0080H         PUBLIC        P0_DR
  D:0090H         PUBLIC        P1_DR
  D:00A0H         PUBLIC        P2_DR
  D:00B0H         PUBLIC        P3_DR
  D:00D0H         PUBLIC        PSW
  -------         PROC          MAIN
  C:0003H         LINE#         31
  C:0003H         LINE#         32
  C:0003H         LINE#         33
  C:0006H         LINE#         34
  C:000CH         LINE#         35
  C:000FH         LINE#         36
  C:0012H         LINE#         37
  C:0026H         LINE#         39
  C:0028H         LINE#         41
  C:0028H         LINE#         42
  C:0028H         LINE#         43
  C:002BH         LINE#         44
  -------         ENDPROC       MAIN
  -------         ENDMOD        MAIN

  -------         MODULE        TOUCH_LIB
  C:0000H         SYMBOL        _ICE_DUMMY_
  C:12CFH         PUBLIC        TKL_ScanStartLoop
  D:001FH         PUBLIC        Touch_Number_sum
  D:00A8H         PUBLIC        IE
  B:0090H.2       PUBLIC        P1_2
  B:0090H.3       PUBLIC        P1_3
  C:11BBH         SYMBOL        _TKL_Key_SetErrorState
  C:0F9AH         SYMBOL        _TKL_Key_SetFindIcomState
  C:002DH         PUBLIC        Delay_Us
  C:0710H         SYMBOL        _TKL_Key_FindIcomTreatment
  C:149EH         PUBLIC        TKL_Action
  C:14E4H         PUBLIC        SDA_OUT
  C:1526H         PUBLIC        I2C_Init
BL51 BANKED LINKER/LOCATER V6.22                                                      08/01/2023  15:50:03  PAGE 8


  C:0AD6H         SYMBOL        _TKL_AddDataToBuf
  C:0036H         PUBLIC        TKL_CSDInit
  D:00E0H         PUBLIC        ACC
  C:153AH         PUBLIC        iic_start
  C:049BH         PUBLIC        _ThresholdInit
  C:0ED1H         SYMBOL        TKL_ProcessAll
  C:155EH         PUBLIC        _Delay_Us1
  C:102CH         PUBLIC        TKL_IRQCallback
  C:14FAH         PUBLIC        SDA_IN
  D:00F8H         PUBLIC        SLPTIM_CR
  C:1420H         PUBLIC        _iic_send_byte
  C:0CFEH         SYMBOL        _TKL_Acquisition
  C:13EBH         PUBLIC        iic_wait_ack
  C:1510H         PUBLIC        iic_stop
  X:0086H         PUBLIC        SendTouch_Number
  C:0BEEH         PUBLIC        _TKL_Init
  C:095DH         SYMBOL        _gpio_set_mode
  C:121AH         PUBLIC        I2C_Write_Buffer
  D:0080H         PUBLIC        P0_DR
  D:0090H         PUBLIC        P1_DR
  C:1452H         SYMBOL        TKL_AcquisitionAll
  D:00A0H         PUBLIC        P2_DR
  D:00B0H         PUBLIC        P3_DR
  D:0021H         PUBLIC        TKLInfo
  C:1148H         SYMBOL        _TKL_Key_SetCalibrationState
  D:00D0H         PUBLIC        PSW
  -------         PROC          SDA_OUT
  C:14E4H         LINE#         187
  C:14E4H         LINE#         188
  C:14E4H         LINE#         189
  C:14EBH         LINE#         190
  C:14F2H         LINE#         191
  C:14F9H         LINE#         192
  -------         ENDPROC       SDA_OUT
  -------         PROC          SDA_IN
  C:14FAH         LINE#         194
  C:14FAH         LINE#         195
  C:14FAH         LINE#         196
  C:1501H         LINE#         197
  C:1508H         LINE#         198
  C:150FH         LINE#         199
  -------         ENDPROC       SDA_IN
  -------         PROC          DELAY_US
  C:002DH         LINE#         202
  C:002DH         LINE#         203
  C:002DH         LINE#         204
  C:002EH         LINE#         205
  C:002FH         LINE#         206
  -------         ENDPROC       DELAY_US
  -------         PROC          _DELAY_US1
  D:0007H         SYMBOL        us
  -------         DO            
  D:0006H         SYMBOL        a
  -------         ENDDO         
  C:155EH         LINE#         208
  C:155EH         LINE#         209
  C:155EH         LINE#         211
BL51 BANKED LINKER/LOCATER V6.22                                                      08/01/2023  15:50:03  PAGE 9


  C:1565H         LINE#         212
  C:1565H         LINE#         213
  C:1566H         LINE#         214
  C:1567H         LINE#         215
  C:1568H         LINE#         217
  C:156BH         LINE#         218
  -------         ENDPROC       _DELAY_US1
  -------         PROC          I2C_INIT
  C:1526H         LINE#         221
  C:1526H         LINE#         222
  C:1526H         LINE#         223
  C:152BH         LINE#         224
  C:152FH         LINE#         225
  C:1535H         LINE#         226
  C:1537H         LINE#         227
  C:1539H         LINE#         228
  -------         ENDPROC       I2C_INIT
  -------         PROC          IIC_START
  C:153AH         LINE#         231
  C:153AH         LINE#         232
  C:153AH         LINE#         233
  C:153DH         LINE#         234
  C:153FH         LINE#         235
  C:1541H         LINE#         236
  C:1546H         LINE#         237
  C:1548H         LINE#         238
  C:154BH         LINE#         239
  C:154DH         LINE#         240
  -------         ENDPROC       IIC_START
  -------         PROC          IIC_STOP
  C:1510H         LINE#         243
  C:1510H         LINE#         244
  C:1510H         LINE#         245
  C:1513H         LINE#         246
  C:1515H         LINE#         247
  C:1517H         LINE#         248
  C:151CH         LINE#         249
  C:151EH         LINE#         250
  C:1521H         LINE#         251
  C:1523H         LINE#         252
  -------         ENDPROC       IIC_STOP
  -------         PROC          IIC_WAIT_ACK
  -------         DO            
  D:0004H         SYMBOL        time
  -------         ENDDO         
  C:13EBH         LINE#         278
  C:13EBH         LINE#         279
  C:13EBH         LINE#         280
  C:13EEH         LINE#         281
  C:13F1H         LINE#         282
  C:13F3H         LINE#         283
  C:13F6H         LINE#         284
  C:13F8H         LINE#         285
  C:13FDH         LINE#         286
  C:1402H         LINE#         287
  C:1402H         LINE#         288
  C:1407H         LINE#         289
BL51 BANKED LINKER/LOCATER V6.22                                                      08/01/2023  15:50:03  PAGE 10


  C:1410H         LINE#         290
  C:1410H         LINE#         291
  C:1413H         LINE#         292
  C:1416H         LINE#         293
  C:1416H         LINE#         294
  C:1416H         LINE#         296
  C:1419H         LINE#         297
  C:141BH         LINE#         298
  C:141DH         LINE#         299
  C:141FH         LINE#         300
  -------         ENDPROC       IIC_WAIT_ACK
  -------         PROC          _IIC_SEND_BYTE
  D:0005H         SYMBOL        dat
  -------         DO            
  D:0004H         SYMBOL        i
  -------         ENDDO         
  C:1420H         LINE#         302
  C:1422H         LINE#         303
  C:1422H         LINE#         305
  C:1425H         LINE#         306
  C:1427H         LINE#         307
  C:1429H         LINE#         308
  C:1429H         LINE#         309
  C:1439H         LINE#         310
  C:143BH         LINE#         311
  C:143FH         LINE#         312
  C:1442H         LINE#         313
  C:1444H         LINE#         314
  C:1449H         LINE#         315
  C:144BH         LINE#         317
  C:144FH         LINE#         318
  -------         ENDPROC       _IIC_SEND_BYTE
  -------         PROC          I2C_WRITE_BUFFER
  -------         DO            
  D:0003H         SYMBOL        Count
  -------         ENDDO         
  C:121AH         LINE#         376
  C:121AH         LINE#         377
  C:121AH         LINE#         379
  C:121DH         LINE#         380
  C:1222H         LINE#         382
  C:1227H         LINE#         383
  C:122CH         LINE#         384
  C:1231H         LINE#         385
  C:1236H         LINE#         386
  C:123BH         LINE#         387
  C:1240H         LINE#         389
  C:1242H         LINE#         390
  C:1242H         LINE#         391
  C:1253H         LINE#         392
  C:1265H         LINE#         393
  C:1269H         LINE#         395
  C:126FH         LINE#         396
  C:1274H         LINE#         398
  -------         ENDPROC       I2C_WRITE_BUFFER
  -------         PROC          TKL_CSDINIT
  C:0036H         LINE#         410
BL51 BANKED LINKER/LOCATER V6.22                                                      08/01/2023  15:50:03  PAGE 11


  C:0036H         LINE#         411
  C:0036H         LINE#         413
  C:003DH         LINE#         414
  C:0042H         LINE#         415
  C:0047H         LINE#         418
  C:004DH         LINE#         419
  C:0053H         LINE#         420
  C:0057H         LINE#         421
  C:005BH         LINE#         426
  -------         ENDPROC       TKL_CSDINIT
  -------         PROC          _THRESHOLDINIT
  D:0019H         SYMBOL        chn
  D:001AH         SYMBOL        cfg
  C:049BH         LINE#         429
  C:04A3H         LINE#         430
  C:04A3H         LINE#         431
  C:04C3H         LINE#         432
  C:04F0H         LINE#         433
  C:0516H         LINE#         435
  C:0537H         LINE#         436
  C:058CH         LINE#         437
  C:05B9H         LINE#         439
  C:060DH         LINE#         440
  C:063AH         LINE#         441
  C:0689H         LINE#         443
  C:069FH         LINE#         444
  C:06B5H         LINE#         446
  C:06C6H         LINE#         447
  C:06D7H         LINE#         449
  C:0705H         LINE#         451
  -------         ENDPROC       _THRESHOLDINIT
  -------         PROC          _TKL_ADDDATATOBUF
  D:001DH         SYMBOL        dat
  C:0AD6H         LINE#         461
  C:0ADAH         LINE#         462
  C:0ADAH         LINE#         464
  C:0ADFH         LINE#         465
  C:0ADFH         LINE#         466
  C:0B49H         LINE#         467
  C:0B49H         LINE#         468
  C:0B75H         LINE#         469
  C:0BA9H         LINE#         472
  C:0BB9H         LINE#         473
  C:0BB9H         LINE#         474
  C:0BD0H         LINE#         476
  C:0BD5H         LINE#         477
  C:0BD5H         LINE#         479
  C:0BD9H         LINE#         480
  C:0BDAH         LINE#         481
  C:0BE3H         LINE#         482
  C:0BE3H         LINE#         484
  C:0BE9H         LINE#         485
  C:0BEDH         LINE#         486
  C:0BEDH         LINE#         487
  C:0BEDH         LINE#         488
  -------         ENDPROC       _TKL_ADDDATATOBUF
  -------         PROC          TKL_SCANSTARTLOOP
BL51 BANKED LINKER/LOCATER V6.22                                                      08/01/2023  15:50:03  PAGE 12


  C:12CFH         LINE#         495
  C:12CFH         LINE#         496
  C:12CFH         LINE#         497
  C:12D7H         LINE#         501
  C:12EEH         LINE#         502
  C:12EEH         LINE#         504
  C:12EEH         LINE#         507
  C:12FEH         LINE#         510
  C:1304H         LINE#         516
  C:130AH         LINE#         517
  C:130FH         LINE#         518
  C:1313H         LINE#         520
  C:1319H         LINE#         525
  C:131FH         LINE#         530
  -------         ENDPROC       TKL_SCANSTARTLOOP
  -------         PROC          TKL_IRQCALLBACK
  C:102CH         LINE#         537
  C:102CH         LINE#         538
  C:102CH         LINE#         540
  C:1032H         LINE#         542
  C:1041H         LINE#         543
  C:1041H         LINE#         545
  C:1048H         LINE#         546
  C:1048H         LINE#         547
  C:1048H         LINE#         548
  C:104BH         LINE#         550
  C:104BH         LINE#         553
  C:1051H         LINE#         556
  C:1053H         LINE#         558
  C:1053H         LINE#         559
  C:1053H         LINE#         560
  C:1056H         LINE#         561
  C:1056H         LINE#         562
  C:1056H         LINE#         563
  C:1059H         LINE#         565
  C:1059H         LINE#         567
  C:1064H         LINE#         570
  C:1085H         LINE#         573
  C:1092H         LINE#         575
  C:10A3H         LINE#         576
  C:10A3H         LINE#         578
  C:10B0H         LINE#         581
  C:10B1H         LINE#         583
  C:10B1H         LINE#         585
  C:10B2H         LINE#         586
  C:10B2H         LINE#         587
  C:10B2H         LINE#         588
  C:10B5H         LINE#         589
  C:10BBH         LINE#         590
  C:10BBH         LINE#         591
  C:10BBH         LINE#         592
  -------         ENDPROC       TKL_IRQCALLBACK
  -------         PROC          _TKL_ACQUISITION
  D:0009H         SYMBOL        Chn
  D:000AH         SYMBOL        pMeasurement
  -------         DO            
  D:000DH         SYMBOL        dat
BL51 BANKED LINKER/LOCATER V6.22                                                      08/01/2023  15:50:03  PAGE 13


  D:000FH         SYMBOL        Max1
  D:0011H         SYMBOL        Max2
  D:0013H         SYMBOL        Min1
  D:0015H         SYMBOL        Min2
  D:0017H         SYMBOL        Sampling
  -------         ENDDO         
  C:0CFEH         LINE#         603
  C:0D06H         LINE#         604
  C:0D06H         LINE#         608
  C:0D19H         LINE#         611
  C:0D1CH         LINE#         612
  C:0D1CH         LINE#         613
  C:0D3FH         LINE#         614
  C:0D48H         LINE#         615
  C:0D48H         LINE#         616
  C:0D4EH         LINE#         617
  C:0D54H         LINE#         618
  C:0D56H         LINE#         619
  C:0D61H         LINE#         620
  C:0D61H         LINE#         621
  C:0D67H         LINE#         622
  C:0D67H         LINE#         623
  C:0D72H         LINE#         624
  C:0D72H         LINE#         625
  C:0D78H         LINE#         626
  C:0D7EH         LINE#         627
  C:0D80H         LINE#         628
  C:0D8BH         LINE#         629
  C:0D8BH         LINE#         630
  C:0D91H         LINE#         631
  C:0D91H         LINE#         632
  C:0D99H         LINE#         633
  C:0DD5H         LINE#         634
  C:0DF5H         LINE#         636
  C:0DF7H         LINE#         637
  -------         ENDPROC       _TKL_ACQUISITION
  -------         PROC          TKL_ACQUISITIONALL
  -------         DO            
  D:0008H         SYMBOL        chn
  -------         ENDDO         
  C:1452H         LINE#         643
  C:1452H         LINE#         644
  C:1452H         LINE#         648
  C:1463H         LINE#         649
  C:1463H         LINE#         650
  C:147FH         LINE#         651
  C:1483H         LINE#         652
  -------         ENDPROC       TKL_ACQUISITIONALL
  -------         PROC          _TKL_KEY_SETFINDICOMSTATE
  D:0019H         SYMBOL        chn
  C:0F9AH         LINE#         660
  C:0F9CH         LINE#         661
  C:0F9CH         LINE#         662
  C:0FB4H         LINE#         663
  C:0FC5H         LINE#         664
  C:0FD7H         LINE#         665
  C:0FDEH         LINE#         666
BL51 BANKED LINKER/LOCATER V6.22                                                      08/01/2023  15:50:03  PAGE 14


  C:0FE6H         LINE#         667
  C:102BH         LINE#         668
  -------         ENDPROC       _TKL_KEY_SETFINDICOMSTATE
  -------         PROC          _TKL_KEY_SETERRORSTATE
  D:000EH         SYMBOL        chn
  C:11BBH         LINE#         675
  C:11BDH         LINE#         676
  C:11BDH         LINE#         677
  C:11D4H         LINE#         678
  C:1219H         LINE#         679
  -------         ENDPROC       _TKL_KEY_SETERRORSTATE
  -------         PROC          _TKL_KEY_SETCALIBRATIONSTATE
  D:000EH         SYMBOL        chn
  C:1148H         LINE#         687
  C:114AH         LINE#         688
  C:114AH         LINE#         689
  C:1161H         LINE#         690
  C:116BH         LINE#         691
  C:1175H         LINE#         692
  C:11BAH         LINE#         693
  -------         ENDPROC       _TKL_KEY_SETCALIBRATIONSTATE
  -------         PROC          _TKL_KEY_FINDICOMTREATMENT
  D:0009H         SYMBOL        chn
  -------         DO            
  D:000AH         SYMBOL        target
  D:000CH         SYMBOL        dat
  -------         ENDDO         
  C:0710H         LINE#         701
  C:0712H         LINE#         702
  C:0712H         LINE#         703
  C:072BH         LINE#         704
  C:072BH         LINE#         705
  C:0741H         LINE#         706
  C:0741H         LINE#         707
  C:075EH         LINE#         708
  C:075EH         LINE#         709
  C:0764H         LINE#         710
  C:0785H         LINE#         729
  C:07A9H         LINE#         730
  C:07A9H         LINE#         731
  C:07B6H         LINE#         732
  C:07B6H         LINE#         733
  C:07DDH         LINE#         734
  C:07DDH         LINE#         735
  C:07EEH         LINE#         736
  C:07F0H         LINE#         738
  C:07F0H         LINE#         739
  C:0808H         LINE#         740
  C:0824H         LINE#         741
  C:0830H         LINE#         742
  C:0830H         LINE#         744
  C:084BH         LINE#         745
  C:084BH         LINE#         746
  C:0850H         LINE#         747
  C:0850H         LINE#         749
  C:0850H         LINE#         750
  C:0853H         LINE#         752
BL51 BANKED LINKER/LOCATER V6.22                                                      08/01/2023  15:50:03  PAGE 15


  C:0853H         LINE#         753
  C:087CH         LINE#         754
  C:087CH         LINE#         755
  C:0890H         LINE#         756
  C:0895H         LINE#         757
  C:0897H         LINE#         759
  C:0897H         LINE#         760
  C:08AFH         LINE#         761
  C:08CBH         LINE#         762
  C:08D7H         LINE#         763
  C:08D7H         LINE#         764
  C:08F2H         LINE#         765
  C:08F2H         LINE#         766
  C:08F7H         LINE#         767
  C:08F7H         LINE#         769
  C:0918H         LINE#         770
  C:0918H         LINE#         771
  C:0918H         LINE#         772
  C:0918H         LINE#         773
  -------         ENDPROC       _TKL_KEY_FINDICOMTREATMENT
  -------         PROC          TKL_PROCESSALL
  -------         DO            
  D:0008H         SYMBOL        chn
  -------         ENDDO         
  C:0ED1H         LINE#         782
  C:0ED1H         LINE#         783
  C:0ED1H         LINE#         786
  C:0ED5H         LINE#         787
  C:0ED5H         LINE#         788
  C:0ED7H         LINE#         789
  C:0ED7H         LINE#         791
  C:0EDAH         LINE#         792
  C:0EDAH         LINE#         793
  C:0EEBH         LINE#         794
  C:0EF2H         LINE#         796
  C:0F03H         LINE#         797
  C:0F03H         LINE#         799
  C:0F1BH         LINE#         800
  C:0F1BH         LINE#         801
  C:0F20H         LINE#         802
  C:0F22H         LINE#         803
  C:0F22H         LINE#         804
  C:0F63H         LINE#         805
  C:0F67H         LINE#         806
  C:0F6CH         LINE#         807
  C:0F6EH         LINE#         808
  C:0F6EH         LINE#         809
  C:0F88H         LINE#         810
  C:0F8FH         LINE#         811
  C:0F97H         LINE#         813
  -------         ENDPROC       TKL_PROCESSALL
  -------         PROC          L?0149
  -------         ENDPROC       L?0149
  -------         PROC          _GPIO_SET_MODE
  D:0007H         SYMBOL        b_PortPin
  D:0005H         SYMBOL        mode
  C:095DH         LINE#         819
BL51 BANKED LINKER/LOCATER V6.22                                                      08/01/2023  15:50:03  PAGE 16


  C:095DH         LINE#         820
  C:095DH         LINE#         821
  C:0965H         LINE#         822
  C:0965H         LINE#         823
  C:096BH         LINE#         824
  C:096BH         LINE#         825
  C:097EH         LINE#         826
  C:0984H         LINE#         827
  C:0987H         LINE#         828
  C:098AH         LINE#         829
  C:0996H         LINE#         830
  C:0996H         LINE#         831
  C:09ADH         LINE#         832
  C:09B3H         LINE#         833
  C:09B6H         LINE#         834
  C:09B8H         LINE#         835
  C:09C4H         LINE#         836
  C:09C4H         LINE#         837
  C:09E1H         LINE#         838
  C:09E7H         LINE#         839
  C:09EAH         LINE#         840
  C:09ECH         LINE#         841
  C:09FEH         LINE#         842
  C:09FEH         LINE#         843
  C:0A15H         LINE#         844
  C:0A1BH         LINE#         845
  C:0A26H         LINE#         846
  C:0A26H         LINE#         847
  C:0A27H         LINE#         848
  C:0A2FH         LINE#         849
  C:0A2FH         LINE#         850
  C:0A35H         LINE#         851
  C:0A35H         LINE#         852
  C:0A49H         LINE#         853
  C:0A4CH         LINE#         854
  C:0A4CH         LINE#         855
  C:0A4FH         LINE#         856
  C:0A5BH         LINE#         857
  C:0A5BH         LINE#         858
  C:0A73H         LINE#         859
  C:0A76H         LINE#         860
  C:0A76H         LINE#         861
  C:0A78H         LINE#         862
  C:0A84H         LINE#         863
  C:0A84H         LINE#         864
  C:0AA2H         LINE#         865
  C:0AA5H         LINE#         866
  C:0AA5H         LINE#         867
  C:0AA7H         LINE#         868
  C:0AB3H         LINE#         869
  C:0AB3H         LINE#         870
  C:0ACBH         LINE#         871
  C:0AD1H         LINE#         872
  C:0AD5H         LINE#         873
  C:0AD5H         LINE#         874
  C:0AD5H         LINE#         875
  -------         ENDPROC       _GPIO_SET_MODE
BL51 BANKED LINKER/LOCATER V6.22                                                      08/01/2023  15:50:03  PAGE 17


  -------         PROC          _TKL_INIT
  D:0008H         SYMBOL        p_TKChnCfg
  D:000BH         SYMBOL        ChnNum
  D:000CH         SYMBOL        ChnInfoPtr
  -------         DO            
  D:000FH         SYMBOL        chn
  D:0010H         SYMBOL        cfg
  -------         ENDDO         
  C:0BEEH         LINE#         884
  C:0BF6H         LINE#         885
  C:0BF6H         LINE#         889
  C:0BF9H         LINE#         891
  C:0C08H         LINE#         892
  C:0C08H         LINE#         894
  C:0C08H         LINE#         897
  C:0C11H         LINE#         898
  C:0C21H         LINE#         899
  C:0C27H         LINE#         901
  C:0C34H         LINE#         902
  C:0C34H         LINE#         903
  C:0C4AH         LINE#         904
  C:0C68H         LINE#         905
  C:0C7EH         LINE#         906
  C:0C9FH         LINE#         907
  C:0CB8H         LINE#         908
  C:0CD7H         LINE#         909
  C:0CE2H         LINE#         910
  C:0CE7H         LINE#         912
  C:0CF1H         LINE#         913
  C:0CF1H         LINE#         914
  C:0CF6H         LINE#         915
  C:0CFAH         LINE#         917
  C:0CFDH         LINE#         918
  -------         ENDPROC       _TKL_INIT
  -------         PROC          TKL_ACTION
  C:149EH         LINE#         924
  C:149EH         LINE#         925
  C:149EH         LINE#         927
  C:14A9H         LINE#         928
  C:14A9H         LINE#         930
  C:14A9H         LINE#         932
  C:14ACH         LINE#         933
  C:14AFH         LINE#         935
  C:14B5H         LINE#         936
  -------         ENDPROC       TKL_ACTION
  -------         ENDMOD        TOUCH_LIB

  -------         MODULE        TOUCHKEYSCAN
  C:0000H         SYMBOL        _ICE_DUMMY_
  D:00A8H         PUBLIC        IE
  C:154EH         PUBLIC        Timer0_Init
  D:0089H         PUBLIC        TMOD
  D:0088H         PUBLIC        TCON
  C:136CH         PUBLIC        Timer0_IRQHandler
  D:00E0H         PUBLIC        ACC
  X:0000H         PUBLIC        ChnInfoBuf
  C:14B6H         PUBLIC        TKChnCfg
BL51 BANKED LINKER/LOCATER V6.22                                                      08/01/2023  15:50:03  PAGE 18


  D:008CH         PUBLIC        TH0
  D:008AH         PUBLIC        TL0
  D:00F8H         PUBLIC        SLPTIM_CR
  C:13B0H         PUBLIC        CSD_IRQHandler
  D:008EH         PUBLIC        CKCON
  D:0080H         PUBLIC        P0_DR
  D:0090H         PUBLIC        P1_DR
  D:00A0H         PUBLIC        P2_DR
  D:00B0H         PUBLIC        P3_DR
  D:00D0H         PUBLIC        PSW
  -------         PROC          TIMER0_IRQHANDLER
  C:136CH         LINE#         12
  C:1389H         LINE#         14
  C:138CH         LINE#         15
  C:138FH         LINE#         16
  C:1392H         LINE#         18
  C:1395H         LINE#         19
  -------         ENDPROC       TIMER0_IRQHANDLER
  -------         PROC          CSD_IRQHANDLER
  C:13B0H         LINE#         21
  C:13CDH         LINE#         23
  C:13D0H         LINE#         24
  -------         ENDPROC       CSD_IRQHANDLER
  -------         PROC          TIMER0_INIT
  C:154EH         LINE#         26
  C:154EH         LINE#         27
  C:154EH         LINE#         28
  C:1551H         LINE#         29
  C:1554H         LINE#         30
  C:1557H         LINE#         31
  C:155AH         LINE#         32
  C:155DH         LINE#         33
  -------         ENDPROC       TIMER0_INIT
  -------         ENDMOD        TOUCHKEYSCAN

  -------         MODULE        ?C?CLDPTR
  C:0066H         PUBLIC        ?C?CLDPTR
  -------         ENDMOD        ?C?CLDPTR

  -------         MODULE        ?C?CLDOPTR
  C:007FH         PUBLIC        ?C?CLDOPTR
  -------         ENDMOD        ?C?CLDOPTR

  -------         MODULE        ?C?CILDOPTR
  C:00ACH         PUBLIC        ?C?CILDOPTR
  -------         ENDMOD        ?C?CILDOPTR

  -------         MODULE        ?C?CSTPTR
  C:00DFH         PUBLIC        ?C?CSTPTR
  -------         ENDMOD        ?C?CSTPTR

  -------         MODULE        ?C?CSTOPTR
  C:00F1H         PUBLIC        ?C?CSTOPTR
  -------         ENDMOD        ?C?CSTOPTR

  -------         MODULE        ?C?SIDIV
  C:0113H         PUBLIC        ?C?SIDIV
BL51 BANKED LINKER/LOCATER V6.22                                                      08/01/2023  15:50:03  PAGE 19


  -------         ENDMOD        ?C?SIDIV

  -------         MODULE        ?C?ILDOPTR
  C:0149H         PUBLIC        ?C?ILDOPTR
  -------         ENDMOD        ?C?ILDOPTR

  -------         MODULE        ?C?ISTPTR
  C:0181H         PUBLIC        ?C?ISTPTR
  -------         ENDMOD        ?C?ISTPTR

  -------         MODULE        ?C?ISTOPTR
  C:01A0H         PUBLIC        ?C?ISTOPTR
  -------         ENDMOD        ?C?ISTOPTR

  -------         MODULE        ?C?ULDIV
  C:0209H         PUBLIC        ?C?ULDIV
  -------         ENDMOD        ?C?ULDIV

  -------         MODULE        ?C?LLDPTR
  C:029BH         PUBLIC        ?C?LLDPTR
  -------         ENDMOD        ?C?LLDPTR

  -------         MODULE        ?C?LLDOPTR
  C:02BBH         PUBLIC        ?C?LLDOPTR
  -------         ENDMOD        ?C?LLDOPTR

  -------         MODULE        ?C?LSTPTR
  C:02EBH         PUBLIC        ?C?LSTPTR
  -------         ENDMOD        ?C?LSTPTR

  -------         MODULE        ?C?LLDPTR0
  C:0305H         PUBLIC        ?C?LLDPTR0
  -------         ENDMOD        ?C?LLDPTR0

  -------         MODULE        ?C?LSTKOPTR
  C:0325H         PUBLIC        ?C?LSTKOPTR
  -------         ENDMOD        ?C?LSTKOPTR

  -------         MODULE        ?C?OFFXADD
  C:0349H         PUBLIC        ?C?OFFXADD
  -------         ENDMOD        ?C?OFFXADD

  -------         MODULE        ?C?UIDIV
  C:0355H         PUBLIC        ?C?UIDIV
  -------         ENDMOD        ?C?UIDIV

  -------         MODULE        ?C?LLDIDATA
  C:03AAH         PUBLIC        ?C?LLDIDATA
  -------         ENDMOD        ?C?LLDIDATA

  -------         MODULE        ?C?LLDXDATA
  C:03B6H         PUBLIC        ?C?LLDXDATA
  -------         ENDMOD        ?C?LLDXDATA

  -------         MODULE        ?C?LLDPDATA
  C:03C2H         PUBLIC        ?C?LLDPDATA
  -------         ENDMOD        ?C?LLDPDATA
BL51 BANKED LINKER/LOCATER V6.22                                                      08/01/2023  15:50:03  PAGE 20



  -------         MODULE        ?C?LLDCODE
  C:03CEH         PUBLIC        ?C?LLDCODE
  -------         ENDMOD        ?C?LLDCODE

  -------         MODULE        ?C?LLDIDATA0
  C:03DEH         PUBLIC        ?C?LLDIDATA0
  -------         ENDMOD        ?C?LLDIDATA0

  -------         MODULE        ?C?LLDXDATA0
  C:03EBH         PUBLIC        ?C?LLDXDATA0
  -------         ENDMOD        ?C?LLDXDATA0

  -------         MODULE        ?C?LLDPDATA0
  C:03F7H         PUBLIC        ?C?LLDPDATA0
  -------         ENDMOD        ?C?LLDPDATA0

  -------         MODULE        ?C?LLDCODE0
  C:0404H         PUBLIC        ?C?LLDCODE0
  -------         ENDMOD        ?C?LLDCODE0

  -------         MODULE        ?C?LSTIDATA
  C:0414H         PUBLIC        ?C?LSTIDATA
  -------         ENDMOD        ?C?LSTIDATA

  -------         MODULE        ?C?LSTXDATA
  C:0420H         PUBLIC        ?C?LSTXDATA
  -------         ENDMOD        ?C?LSTXDATA

  -------         MODULE        ?C?LSTPDATA
  C:042CH         PUBLIC        ?C?LSTPDATA
  -------         ENDMOD        ?C?LSTPDATA

  -------         MODULE        ?C?LSTKIDATA
  C:0438H         PUBLIC        ?C?LSTKIDATA
  -------         ENDMOD        ?C?LSTKIDATA

  -------         MODULE        ?C?LSTKXDATA
  C:0451H         PUBLIC        ?C?LSTKXDATA
  -------         ENDMOD        ?C?LSTKXDATA

  -------         MODULE        ?C?LSTKPDATA
  C:0482H         PUBLIC        ?C?LSTKPDATA
  -------         ENDMOD        ?C?LSTKPDATA

Program Size: data=52.0 xdata=184 code=5474
LINK/LOCATE RUN COMPLETE.  0 WARNING(S),  0 ERROR(S)
